S113D000183C36C1FF2747C1002715C105272AC18F
S113D010042204C101242FBDD05A2000321838390B
S113D020C63FBDD0F8BDD0F8C60FBDD0F8C606BD0A
S113D030D0F8C601BDD0F820E3BDD106BDD0B418E8
S113D0403018A70020D6BDD0D6BDD0AB20CEE60088
S113D050C10427C8BDD05F0820F4C104260139C12A
S113D0600D2604BDD07139BDD0FFBDD106BDD07829
S113D07039BDD106BDD089398114272381402727A2
S113D0808154271F810027113981132312812723FB
S113D090168153230E8167230086018080200C862D
S113D0A040200886142004865420003716CB80BD07
S113D0B0D0F8333981132204C601201881272206AF
S113D0C0C6038014200E81532206C6028040200429
S113D0D0C60480544C398100270781142302860139
S113D0E04AC1012712C10226048B40200AC103262B
S113D0F0048B1420028B5439F72000BDD11439F766
S113D1003000BDD1143918CE0002B620002BFB1814
S110D1100926F73918CE0800180926FC3945
S105FFF2C01C2D
S113C0008642B71002863FB710097F10070E8620BC
S113C010B7100846CEC0000926FD20F4CE10001F3C
S113C02002800FB61002B61005B71004B70015BD94
S106C030E0843B6A
S105001A0D04CF
S113E00048657420676574616C20046C69677420CA
S113E010696E2068657420696E74657276616C043B
S113E0203C2E2E2E2C2D32303E045B2D32302C2DE6
S113E03031353E045B2D31352C2D31303E045B2DC2
S113E04031302C2D20353E045B2D20352C2D2030F5
S113E0503E045B2020302C2020353E045B202035FC
S113E0602C2031303E045B2031302C2031353E04ED
S113E0705B2031352C2032303E045B2032302C2E94
S113E0802E2E3E049615BDE0D286EC971C7F001D13
S113E0909615911C2D0F961C8B05971C7C001D96C4
S113E0A01D810925EBC600BDD000CEE000C6FFBD32
S113E0B0D000CE0016C6FFBDD000CEE00BC6FFBD1B
S113E0C0D000CEE020961DC60A3D3AC6FFBDD00062
S113E0D00139862BD6152A03862D50971686304C87
S113E0E0C06424FBCB644A971786304CC00A24FBD7
S10DE0F0CB0A4A9718CB30D7193930
S9030000FC
